:03000000021E4E8F
:101E4E0075C7AA75C75575FD5A75C7AA75C7557555
:101E5E00FDA5787FE4F6D8FD9000007FFF7E03E4B9
:0C1E6E00F0A3DFFCDEFA758121021EB536
:10246F009001DB120ADE538EF7438901D28C7F0075
:10247F007E007D007C009001DBE0F8A3E0F9A3E093
:10248F00FAA3E0FBC3120ABA6035758A7E758CFF1A
:10249F00308DFDC28D9001DBE0FCA3E0FDA3E0FEDB
:1024AF00A3E0FF7BFF7AFF79FF78FFEF2BFFEE3A78
:1024BF00FEED39FDEC38FC9001DB120ADE80AFC275
:0224CF008C225D
:1024D1009001DF120ADE538EF7438901D28C7F000F
:1024E1007E007D007C009001DFE0F8A3E0F9A3E02D
:1024F100FAA3E0FBC3120ABA6035758ACA758CFA71
:10250100308DFDC28D9001DFE0FCA3E0FDA3E0FE74
:10251100A3E0FF7BFF7AFF79FF78FFEF2BFFEE3A15
:10252100FEED39FDEC38FC9001DF120ADE80AFC20E
:022531008C22FA
:102533009001E3120ADE538EEF438910D28E7F009F
:102543007E007D007C009001E3E0F8A3E0F9A3E0C6
:10255300FAA3E0FBC3120ABA6035758BEA758DCB1B
:10256300308FFDC28F9001E3E0FCA3E0FDA3E0FE0A
:10257300A3E0FF7BFF7AFF79FF78FFEF2BFFEE3AB3
:10258300FEED39FDEC38FC9001E3120ADE80AFC2A8
:022593008E2296
:10227A009001E7120ADE53C9BF53C9DF43C910D21E
:10228A00CA7F007E007D007C009001E7E0F8A3E0B1
:10229A00F9A3E0FAA3E0FBC3120ABA603575CC30A1
:1022AA0075CDF830CFFDC2CF9001E7E0FCA3E0FD89
:1022BA00A3E0FEA3E0FF7BFF7AFF79FF78FFEF2B15
:1022CA00FFEE3AFEED39FDEC38FC9001E7120ADE2A
:0522DA0080AFC2CA2222
:1022DF009001EB120ADE75C40743C4087F007E002D
:1022EF007D007C009001EBE0F8A3E0F9A3E0FAA3F6
:1022FF00E0FBC3120ABA603875C52C75C6CFE5C4AA
:10230F0030E4FB53C4EF9001EBE0FCA3E0FDA3E04E
:10231F00FEA3E0FF7BFF7AFF79FF78FFEF2BFFEE45
:10232F003AFEED39FDEC38FC9001EB120ADE80AC81
:04233F0053C4F7226A
:102343009001EF120ADE75C40243C4087F007E00C9
:102353007D007C009001EFE0F8A3E0F9A3E0FAA38D
:10236300E0FBC3120ABA603875C5D875C6FFE5C469
:1023730030E4FB53C4EF9001EFE0FCA3E0FDA3E0E6
:10238300FEA3E0FF7BFF7AFF79FF78FFEF2BFFEEE1
:102393003AFEED39FDEC38FC9001EF120ADE80AC19
:0423A30053C4F72206
:1023A7009001F3120ADE75C40243C4087F007E0061
:1023B7007D007C009001F3E0F8A3E0F9A3E0FAA325
:1023C700E0FBC3120ABA603875C5FC75C6FFE5C4E1
:1023D70030E4FB53C4EF9001F3E0FCA3E0FDA3E07E
:1023E700FEA3E0FF7BFF7AFF79FF78FFEF2BFFEE7D
:1023F7003AFEED39FDEC38FC9001F3120ADE80ACB1
:0424070053C4F722A1
:10240B009001F7120ADE75C40243C4087F007E00F8
:10241B007D007C009001F7E0F8A3E0F9A3E0FAA3BC
:10242B00E0FBC3120ABA603875C56075C6F0E5C427
:10243B0030E4FB53C4EF9001F7E0FCA3E0FDA3E015
:10244B00FEA3E0FF7BFF7AFF79FF78FFEF2BFFEE18
:10245B003AFEED39FDEC38FC9001F7120ADE80AC48
:04246B0053C4F7223D
:0C2882004401860000000042018A0000B2
:03000B0002136578
:10136500C0E0C0F0C083C082C0D075D000C000C04E
:1013750001C002C003C004C005C006C00790020D2D
:10138500E0FEA3E0FFEEFF7E008F8C90020DE0FEF5
:10139500A3E0FFEF54FFF58A900186E0FCA3E0FD92
:1013A500A3E0FEA3E0FFEF2401FFEE3400FEED34E1
:1013B50000FDEC3400FC900186120ADE7F007E5CA5
:1013C5007D267C05900186E0F8A3E0F9A3E0FAA369
:1013D500E0FBC3120ABA400A900186120AEA00002D
:1013E500000090018BE004F0700690018AE004F0A3
:1013F50090018AE0FEA3E0FFEF20E00E90018CE073
:10140500FFEF4401FF90018CEFF090018AE0FEA30D
:10141500E0FF7C007D0A1208F0ED4C700E90018C07
:10142500E0FFEF4402FF90018CEFF090018AE0FEAF
:10143500A3E0FF7C007D141208F0ED4C70119001C3
:101445008CE0FFEF4404FF90018CEFF0121A3F90FF
:10145500018AE0FEA3E0FF7C007D641208F0ED4CFC
:10146500700E90018CE0FFEF4408FF90018CEFF0C7
:1014750090018AE0FEA3E0FF7C007DC81208F0ED34
:101485004C700E90018CE0FFEF4410FF90018CEF43
:10149500F090018AE0FEA3E0FF7C017DF41208F0E4
:1014A500ED4C700E90018CE0FFEF4420FF90018C15
:1014B500EFF090018AE0FEA3E0FF7C037DE81208CF
:1014C500F0ED4C700E90018CE0FFEF4440FF900171
:1014D5008CEFF090018AE0FEA3E0FF7C137D88127B
:1014E50008F0ED4C701690018CE0FFEF4480FF9002
:1014F500018CEFF090018AE4F0A3E4F0D007D00668
:10150500D005D004D003D002D001D000D0D0D082F5
:07151500D083D0F0D0E032DA
:03001B00020007D9
:0100070032C6
:1027F8009001FB120ADE53B1BF53B2BF53B17F53EE
:10280800B27F759850438920438780438E1053C404
:10281800DF9001FBE0F8A3E0F9A3E0FAA3E0FB7F77
:10282800407E427D0F7C00120A12EF04FFEFF40491
:07283800F58DD28ED299222A
:101EFA009001FF120ADE53B1BF53B2BF53B17F53F1
:101F0A00B27F75985043878053C4F843C420900128
:101F1A00FFE0F8A3E0F9A3E0FAA3E0FB7F407E42EA
:101F2A007D0F7C00120A12A804A905AA06AB07C3F2
:101F3A0074FF9BFF74FF9AFEE499FDE498FC78080D
:101F4A00120ACB8FC69001FFE0F8A3E0F9A3E0FAEA
:101F5A00A3E0FB7F407E427D0F7C00120A12A80498
:101F6A00A905AA06AB07C374FF9BFF74FF9AFEE498
:101F7A0099FDE498FCEF54FFFFEE5400FEED540087
:0D1F8A00FDEC5400FC8FC543C408D2992221
:102A6E003098FD90021EE599F0C29890021EE0FF8C
:012A7E002235
:102A4A0090021FEFF0C29990021FE0FF8F99309910
:022A5A00FD225B
:101F9700900203120ADE53B1FB53B2FB53B3BF5394
:101FA700B4BF75F85075C40853C4DF900203E0F856
:101FB700A3E0F9A3E0FAA3E0FB7F407E427D0F7C1C
:101FC70000120A12A804A905AA06AB07C374FF9B4F
:101FD700FF74FF9AFEE499FDE498FC7808120ACB97
:101FE7008FC6900203E0F8A3E0F9A3E0FAA3E0FBB1
:101FF7007F407E427D0F7C00120A12A804A905AA21
:1020070006AB07C374FF9BFF74FF9AFEE499FDE4D8
:1020170098FCEF54FFFFEE5400FEED5400FDEC5426
:0820270000FC8FC543C4082230
:102A7F0030F8FD900220E59AF0C2F8900220E0FFB6
:012A8F002224
:102A5C00900221EFF0C2F9900221E0FF8F9A30F939
:022A6C00FD2249
:102655009001B4EBF0A3EAF0A3E9F09001B7EDF037
:102665009001B9E4F09001B8E4F09001B7E0FF9073
:1026750001B8E0FEEEC39F502E9001B9E0FF900136
:10268500B4E0FBA3E0FAA3E0F99001B8E0FE8E8286
:1026950075830012087DFEEF6EFF9001B9EFF09093
:0C26A50001B8E004F080C39001B9E0FF30
:0126B1002206
:10151C0090017DEBF0A3EAF0A3E9F0900180EDF0EF
:10152C00900184E4F0900180E0FFEF14FF900184BF
:10153C00E0FEEEC39F40030216B190017DE0FBA3D9
:10154C00E0FAA3E0F9900184E0FF8F82758300122A
:10155C00087DFFEF64AA60030216A8900184E0FFE7
:10156C00900180E0FEC3EE9FFFEFC3940450030292
:10157C0016A8900184E0FF7E00EF2401FFEE3400FA
:10158C00FE90017DE0FBA3E0FAA3E0F98F828E834D
:10159C0012087DFF900185EFF0900185E0FF7E0041
:1015AC00900184E0FD7C00ED2FFFEC3EFEEF240368
:1015BC00FFEE3400FE90017DE0FBA3E0FAA3E0F91E
:1015CC008F828E8312087DFFEF64BB60030216A826
:1015DC0090017DE0FBA3E0FAA3E0F9900184E0FF29
:1015EC007E00E92FF9EA3EFAC003C002C001900167
:1015FC0081E0FBA3E0FAA3E0F9120B3B900185E03C
:10160C00FF7E00EF2404FFEE3400FE900181E0FB2E
:10161C00A3E0FAA3E0F9758203758300EE8FF01254
:10162C0009A9900181E0FBA3E0FAA3E0F9120B1BDE
:10163C00E92402F9EA3400FAC003C002C0019001A7
:10164C0081E0FBA3E0FAA3E0F97582037583001235
:10165C000971FFAEF0EF24FCFDD001D002D00312D3
:10166C002655900185E0FEEEFD7C00900184E0FEA5
:10167C00EEFB7A00EB2DFDEA3CFCED2402FDEC3494
:10168C0000FC90017DE0FBA3E0FAA3E0F98D828CD5
:10169C008312087DFEEFB506037F0122900184E0E2
:0716AC0004F00215317F007C
:0116B3002214
:10192E0090018EEBF0A3EAF0A3E9F0900191EDF0B7
:10193E00900191E0FFEFC3942E4003021A3C9000F9
:10194E00E874AAF0900191E0FF9000E9EFF09001A9
:10195E0095E4F0900191E0FF900195E0FEEEC39FBB
:10196E00503290018EE0FBA3E0FAA3E0F9900195CE
:10197E00E0FF8F8275830012087DFF900195E0FED7
:10198E0074EA2EF582E43400F583EFF0900195E0D1
:10199E0004F080BF90018EE0FBA3E0FAA3E0F99083
:1019AE000191E0FD122655900195E0FE74EA2EF5A8
:1019BE0082E43400F583EFF0900195E0FF74EB2F95
:1019CE00F582E43400F58374BBF0900195E4F09059
:1019DE000191E0FF7E00EF2404FFEE3400FE900143
:1019EE0095E0FD7C00C3ED9FEE6480F8EC6480987A
:1019FE005032900195E0FF74E82FF582E43400F543
:101A0E0083E0FF900192E0FBA3E0FAA3E0F99001DE
:101A1E0095E0FE8E82758300EF1208BC900195E072
:101A2E0004F080AB900191E0FFEF2404FF227F00D1
:011A3E002285
:10220F00900222EFF0900222E0FFEFC39401405AB8
:10221F00900222E0FFEFD39431400122900222E09E
:10222F00FF7E007C3E7D801208DE7C007D0C120854
:10223F00F0C3E49FFFE49EFE90020DEEF0A3EFF0DB
:10224F005389F0438901538EF790020DE0FEA3E00E
:10225F00FFEEFF7E008F8C90020DE0FEA3E0FFEFFC
:0B226F0054FFF58AD2A9D2AFD28C2216
:08292F00900207EEF0A3EFF0A7
:10293700900207E0FEA3E0FF8F828E83E493FE748C
:102947000193FFEEFF7E00900209EFF0900209E08D
:01295700FF80
:01295800225C
:0D114A00900196EEF0A3EFF0900198EDF00B
:10115700900199E4F0900196E0FEA3E0FFEF780795
:10116700CEC313CE13D8F9FFEF7807C333CE33CEF0
:10117700D8F9FF90019AEEF0A3EFF0900199E4F00F
:10118700900199E0FFEFC394805043900199E0FFED
:101197007E0090019AE0FCA3E0FDEF2DFFEE3CFE00
:1011A70012292F7E0090019CEEF0A3EFF090019C96
:1011B700E0FEA3E0FF900199E0FE74002EF582E4C3
:1011C7003400F583EFF0900199E004F080B29001CC
:1011D70098E0FF900196E0FCA3E0FD7C00ED547FD2
:1011E700FD74002DF58274003CF583EFF090019AB1
:1011F700E0FEA3E0FFEF54FFF5A690019AE0FEA3FF
:10120700E0FFEEFF7E00EF54FFF5A775AEFFA2AF3C
:10121700E433FF90021DEFF0C2AF75C7AA75C7553B
:10122700439F0190021DE0FFEF24FF92AFA2AFE4BE
:1012370033FF90021DEFF0C2AF75C7AA75C75543BC
:10124700A50190021DE0FFEF24FF92AF75AF22A228
:10125700AFE433FF90021DEFF0C2AF75C7AA75C7A1
:101267005543A40190021DE0FFEF24FF92AFA2AF08
:10127700E433FF90021DEFF0C2AF75C7AA75C755DB
:10128700439F0190021DE0FFEF24FF92AFA2AFE45E
:1012970033FF90021DEFF0C2AF75C7AA75C755435C
:1012A700A50190021DE0FFEF24FF92AF75AF2190DB
:1012B7000199E4F0900199E0FFEFC39480506090AA
:1012C700019AE0FEA3E0FFEF54FFFF900199E0FED3
:1012D700EF2EF5A690019AE0FEA3E0FFEEFF7E0059
:1012E700EF54FFF5A7900199E0FF74002FF582E412
:1012F7003400F583E0FF8FAEA2AFE433FF90021D09
:10130700EFF0C2AF75C7AA75C75543A40190021D78
:10131700E0FFEF24FF92AF900199E004F08095A2DF
:10132700AFE433FF90021DEFF0C2AF75C7AA75C7D0
:101337005553A5FE90021DE0FFEF24FF92AFA2AF29
:10134700E433FF90021DEFF0C2AF75C7AA75C7550A
:0D135700539FFE90021DE0FFEF24FF92AFB8
:011364002266
:0A000E0011223344550000000000E9
:10288E004501780040484A514501730040484A517D
:0529F30090020FEFF05F
:1029F800900210E4F090020FE0FF900210E0FEEE6B
:0D2A0800C39F500900900210E004F080E828
:012A1500229E
:0528F700900211EFF05A
:1028FC00900211E0FF8FF5900212E4F0900212E0CA
:10290C00FFEFC394FF500DE5F420E708900212E0AE
:10291C0004F080E853F47F900211E5F5F090021179
:02292C00E0FFCA
:01292E002286
:0A29590090020AEFF090020BEDF07F
:10296300C29590020AE0FF1228F790020CEFF09054
:0E297300020BE0FF1228F7D29590020CE0FF55
:012981002233
:052A1600900213EFF037
:102A1B00C295900213E0FF1228F77FFF1228F79060
:0B2A2B000214EFF0D295900214E0FFBF
:012A3600227D
:102595009001A6EFF09001A7EBF0A3EAF0A3E9F014
:1025A500C2959001A6E0FF1228F79001ABEFF090DD
:1025B50001ACE4F09001AAE0FF9001ACE0FEEEC3AF
:1025C5009F50267FFF1228F79001A7E0FBA3E0FAB2
:1025D500A3E0F99001ACE0FE8E82758300EF12084E
:1025E500BC9001ACE004F080CBD2959001ABE0FF4C
:0125F50022C3
:1026B2009001ADEFF09001AEEBF0A3EAF0A3E9F0E8
:1026C200C2959001ADE0FF1228F79001B2EFF090B1
:1026D20001B3E4F09001B1E0FF9001B3E0FEEEC37C
:1026E2009F501F9001AEE0FBA3E475F00112095B5D
:1026F200A9F0FA120864FF1228F79001B3E004F07F
:0927020080D2D2959001B2E0FFF3
:01270B0022AB
:10202F009001BAEBF0A3EAF0A3E9F09001BDEDF057
:10203F009001BFE4F07F07122A169001BEEFF090D7
:10204F0001BEE0FFEF30E6539001BEE0FFEF54BF5B
:10205F00FF9001BEEFF0C2919001BDE0FFEFC3947E
:10206F002050079001BDE0FF80027F209001BDEF5F
:10207F00F09001BAE0FBA3E0FAA3E0F99001AA7493
:10208F0020F07F611225957DFF7FE2122959D291B1
:10209F007F961229F39001BF7401F09001BEE0FD0D
:0A20AF007F271229599001BFE0FFBE
:0120B9002204
:101B1E0090019EEBF0A3EAF0A3E9F09001A1EDF0A5
:101B2E009001A27401F0C2919001A1E0FFEFC39465
:101B3E002050079001A1E0FF80027F209001A1EFCD
:101B4E00F090019EE0FBA3E0FAA3E0F99001B174DE
:101B5E0020F07FA01226B2D2919001A4E4F0A3E46B
:101B6E00F09001A4E0FEA3E0FFE4FCFD7BFF7AFF12
:101B7E0079007800D3120AA440132083109001A597
:101B8E00E004F070069001A4E004F080D47F071208
:101B9E002A169001A3EFF09001A3E0FFEF30E41AB4
:101BAE007DFF7FE11229599001A3E0FFEF54EFFF73
:101BBE009001A3EFF09001A2E4F09001A3E0FFEFFB
:101BCE0030E5139001A3E0FFEF54DFFF9001A3EF88
:101BDE00F09001A2E4F09001A3E0FD7F27122959B5
:051BEE009001A2E0FFE0
:011BF30022CF
:101D9E0090015DE4F07BFF7A00790EC003C002C0B3
:101DAE00017B017A01795EA801AC02AD03D001D0AE
:101DBE0002D0037E007F0512083E7BFF7A00791366
:101DCE00C003C002C0017B017A017963A801AC0295
:101DDE00AD03D001D002D0037E007F0512083EC2B3
:101DEE0090D295C2917B017A01795E9001B1740512
:101DFE00F07F301226B27B017A0179639001AA74CA
:101E0E0005F07F10122595900163E0FFEFB4112AC3
:101E1E00900164E0FFEFB42221900165E0FFEFB482
:101E2E003318900166E0FFEFB4440F900167E0FFB6
:0F1E3E00EFB4550690015D7401F090015DE0FF77
:011E4D002272
:10283F00900215E4F0A3E4F0900215E0FEA3E0FF90
:10284F00C3EF9432EE94005021121D9EEF701B7F48
:10285F000A7E007D007C00122343900216E004F0F4
:10286F007006900215E004F080CE900215E0FEA3F2
:02287F00E0FF78
:012881002234
:10213500C2917D207F311229597DFF7FE2122959F5
:102145007B017A0179789001B17405F07F30122610
:10215500B27B017A0179739001B17405F07F2A127F
:1021650026B27D057F211229597D017F2212295929
:102175007D007F3D1229597D017F3C1229597D1A29
:102185007F241229597D287F251229597D0F7F2605
:0D2195001229597D0F7F20122959D2912265
:1027AF009001CCEBF0A3EAF0A3E9F09001CFEDF0AC
:1027BF00C2917D0E7F20122959D2917F0F1229F3DA
:1027CF009001CCE0FBA3E0FAA3E0F99001CFE0FD8C
:1027DF00121B1E9001D0EFF0C2917D0F7F201229A6
:0827EF0059D2919001D0E0FFE6
:0127F70022BF
:04289E004101C5002F
:0100080022D5
:0100090022D4
:1021A200120009C2B07F147E007D007C0012240B55
:1021B200D2B07F1E7E007D007C001223A712000891
:1021C2009001C5E4F020B01D9001C5E004FFF0EFDE
:1021D200D3945040037F00227F017E007D007C006B
:1021E2001223A780E09001C5E4F030B01D9001C534
:1021F200E004FFF0EFD3945040037F00227F017E82
:0D220200007D007C001223A780E07F0122F8
:101CCA0090021874FFF030B003021D98900217E4D6
:101CDA00F0900217E0FFEFC394084003021D9890AA
:101CEA0001C5E4F020B0209001C5E004FFF0EFD375
:101CFA0094324006900218E0FF227F017E007D00A8
:101D0A007C001223A780DD9001C5E4F030B020905A
:101D1A0001C5E004FFF0EFD394504006900218E0AA
:101D2A00FF227F017E007D007C001223A780DD90C8
:101D3A0001C5E0FFEFD394254025900218E0FF90FB
:101D4A000217E0FEC374079EFE7401A8060880020B
:101D5A00C333D8FCFEEF4EFF900218EFF0802690B6
:101D6A000218E0FF900217E0FEC374079EFE74019A
:101D7A00A806088002C333D8FCFEEEF4FEEF5EFF2D
:101D8A00900218EFF0900217E004F0021CDB9002B8
:031D9A0018E0FF4F
:011D9D002223
:0B1814009001D1EBF0A3EAF0A3E9F093
:10181F001221A2EF7003021923121CCA9001D1E00A
:10182F00FBA3E0FAA3E0F9EF1208AA121CCA900179
:10183F00D1E0FBA3E0FAA3E0F9758201758300EF15
:10184F001208BC121CCA9001D1E0FBA3E0FAA3E07E
:10185F00F9758202758300EF1208BC121CCA900141
:10186F00D1E0FBA3E0FAA3E0F9758203758300EFE3
:10187F001208BC121CCA9001D1E0FBA3E0FAA3E04E
:10188F00F9758204758300EF1208BC9001D1E0FB5B
:10189F00A3E0FAA3E0F975820175830012087DFFBA
:1018AF009001D1E0FBA3E0FAA3E0F9120864FEEE89
:1018BF002FFF9001D1E0FBA3E0FAA3E0F9758202BC
:1018CF0075830012087DFEEF2EFF9001D1E0FBA380
:1018DF00E0FAA3E0F975820375830012087DFEEF2D
:1018EF002EFF9001D5EFF09001D1E0FBA3E0FAA31A
:1018FF00E0F975820475830012087DFF9001D5E031
:10190F00FEEFB506089001D47401F0800C9001D45D
:0E191F00E4F080059001D4E4F09001D4E0FFE4
:01192D002297
:0E28A2004B016800FF2A9F00000000000000AC
:0A2A9F002097047F0180027F0022CF
:101A3F00900223E4F0900223E0FFEFC394014003F0
:101A4F00021B1D900223E0FFEF75F00BA42469F534
:101A5F0082E43401F583E0FBA3E0FAA3E0F9120B73
:101A6F00B0EF7003021AFC900223E0FFEF75F00B4A
:101A7F00A4246DF582E43401F583E475F0011209B5
:101A8F0045900223E0FFEF75F00BA4246DF582E47F
:101A9F003401F583E0FEA3E0FFEF64044E7018906D
:101AAF000223E0FFEF75F00BA42472F582E43401FA
:101ABF00F5837401F0804E900223E0FFEF75F00B79
:101ACF00A4246DF582E43401F583E0FEA3E0FFEF7B
:101ADF00647D4E7030900223E0FFEF75F00BA4246D
:101AEF0072F582E43401F5837404F08018900223B8
:101AFF00E0FFEF75F00BA4246DF582E43401F5835C
:0E1B0F00E4F0A3E4F0900223E004F0021A4494
:011B1D0022A5
:1029CF00900172E0FFEFB40109900172E4F0120080
:1029DF001822900172E0FFEFB40408900172E4F046
:0429EF0012001A2296
:01000A0022D3
:0100180022C5
:0100190022C4
:01001A0022C3
:012AA900220A
:101BF4000A535049206572726F722E0A000A536CA0
:101C04006176652052657475726E202563210A0021
:101C14000A486F6D65204C696768742025732C2011
:101C24004275696C64206279204B696E766520691F
:101C34006E20256C640A0056312E30005549443D0F
:101C440025782578257825780A004E524632344C7A
:101C5400303120696E6974204F4B210A0053656E40
:101C6400643A2025730A00253032642525202D206E
:101C740025303264430A00526563763A2025730A9C
:101C8400003E313233343536373839300000000005
:101C94000000000000000000000000000000000040
:101CA4000000000000000000000000000000000030
:101CB4000000000000000000000000000000000020
:061CC4000000000000001A
:0C28B00041014F0041014E0041015C005D
:1029A9007BFF7A1B79F4120E50D2877FF47E017D6A
:1029B900007C001224D1C2877FF47E017D007C0057
:0629C9001224D180E4227B
:1028BD0053F3BF53B3DF53B4DF53B3FE53B4FE53DF
:1028CD00B1FE53B2FE53B1FD53B2FD43F40853F3C1
:1028DD007F53F3DF53F3F753F3FB43F31043F3014C
:0A28ED0053F3FD43F34053F47F2240
:1016B4009001C6EBF0A3EAF0A3E9F0C29575F590AA
:1016C4007F017E007D007C00122343E5F430E7FBBC
:1016D40053F47FE5F5644E60031229A97BFF7A1C5D
:1016E400790190011DE5F5F0120E5075F5017F01A9
:1016F4007E007D007C00122343E5F430E7FB53F4C5
:101704007FE5F5645560031229A97BFF7A1C7901F2
:1017140090011DE5F5F0120E5075F5027F017E0073
:101724007D007C00122343E5F430E7FB53F47FE5AE
:10173400F5645660031229A97BFF7A1C7901900194
:101744001DE5F5F0120E5075F5037F017E007D0056
:101754007C00122343E5F430E7FB53F47FE5F564A2
:101764004F60031229A97BFF7A1C790190011DE5C2
:10177400F5F0120E5075F5047F017E007D007C00AB
:10178400122343E5F430E7FB53F47FE5F56454603A
:10179400031229A97BFF7A1C790190011DE5F5F05C
:1017A400120E5075F5FF7F017E007D007C00122330
:1017B40043E5F430E7FB53F47F9001C6E0FBA3E07C
:1017C400FAA3E0F9E5F51208AA7BFF7A1C790190E7
:1017D400011DE5F5F0120E5075F5FF7F017E007DC9
:1017E400007C00122343E5F430E7FB53F47F9001BF
:1017F400C9E0FBA3E0FAA3E0F9E5F51208AA7BFF30
:101804007A1C790190011DE5F5F0120E50D2952253
:102A370075C7AA75C75575FD5A75C7AA75C7557560
:032A4700FDA522C8
:0400030053A37F2262
:1025F600900224E4F0E58730E4095387EF90022443
:102606007401F0E5A330E10953A3FD90022474029E
:10261600F0E5A230E60953A2BF9002247403F0E568
:10262600A230E50953A2DF9002247404F0E5AA3033
:10263600E30953AAF79002247405F0E5A230E709EE
:0E26460053A27F9002247406F0900224E0FF5D
:012654002263
:0F2A900053A27FC2AF75C7AA75C755439F802257
:05275E00900219EFF0EC
:1027630090021AE4F0900219E0FF90021AE0FEEEE4
:10277300C39F502D900219E0FFEFC394055022D25E
:10278300927F017E007D007C001222DFC2927F01D6
:102793007E007D007C001222DF90021AE004F080AC
:0B27A300C4A292E433FF90014FEFF05E
:0127AE002208
:0520BA0090021BEFF095
:1020BF00A2AFE433FF90021DEFF0C2AF75C7AA7550
:1020CF00C755439F0190021DE0FFEF24FF92AF9091
:1020DF00021BE0FF8FA675A70075AF04A2AFE43314
:1020EF00FF90021DEFF0C2AF75C7AA75C75543A485
:1020FF000190021DE0FFEF24FF92AF90021CE5AEAE
:10210F00F0A2AFE433FF90021DEFF0C2AF75C7AA84
:10211F0075C755539FFE90021DE0FFEF24FF92AF4E
:05212F0090021CE0FF1E
:012134002288
:10270C009001D6EFF09001D7EBF0A3EAF0A3E9F03B
:10271C009001DAE4F09001DAE0FFEFC3940C503151
:10272C009001D6E0FF9001DAE0FEEE2FFF1220BA06
:10273C009001D7E0FBA3E0FAA3E0F99001DAE0FE08
:10274C008E82758300EF1208BC9001DAE004F080F1
:01275C00C4B8
:01275D002259
:10001E007BFF7A1C7985C003C002C0017B017A0088
:10002E007982A801AC02AD03D001D002D0037E00CC
:10003E007F2012083E7BFF7A1C79A5C003C002C048
:10004E00017B017A0079A2A801AC02AD03D001D0E8
:10005E0002D0037E007F2012083E7BFF7A1C79C5FA
:10006E00C003C002C0017B017A0079E2A801AC0294
:10007E00AD03D001D002D0037E007F0512083E9062
:10008E0000E7E4F01225F6900080EFF0122A371206
:10009E00000375B10075B20075B30075B40075AC90
:1000AE000075AD007F0112220F7F007EC27D017CA4
:1000BE00001227F87FE87E037D007C001223437B2D
:1000CE00FF7A1C7914C003C002C0017BFF7A1C7931
:1000DE003B90011DEBF0A3EAF0A3E9F09001201292
:1000EE000AEA6BD7BE99D001D002D003120E507B14
:1000FE00017A0179427F0012270C7BFF7A1C79402E
:10010E00900142E0FF90011DEFF0900143E0FF905F
:10011E00011EEFF0900144E0FF90011FEFF09001FF
:10012E0045E0FF900120EFF0120E50900081E4F0B8
:10013E00900081E0FFEFC3940C502B900081E0FF04
:10014E007E00EF2481FFEE3438FE12292F900081BD
:10015E00E0FE74502EF582E43401F583EFF090004A
:10016E0081E004F080CA7F017E007D007C001222B7
:10017E00DF900172E0FFEFB4010B900172E4F0909A
:10018E00015C7401F01228BD12283F1221357BFF4D
:10019E007A1C794E120E5090015CE0FFEF120B8A22
:1001AE0002DA0001B801000002DA90018CE0FFEFE4
:1001BE0030E42B90018CE0FFEF54EFFF90018CEFB9
:1001CE00F090014FE0FFEF70047F0180027F0090FE
:1001DE00014FEFF090014FE0FFEF24FF929290015C
:1001EE0072E0FFEF64017079900172E4F07E007F9F
:1001FE00207D007B017A007982120D60900082745E
:10020E002AF0900083743FF07B017A007982C0035C
:10021E00C002C0017B017A0079C2900192EBF0A37B
:10022E00EAF0A3E9F0D001D002D0037D0212192E1C
:10023E007B017A0079C27D201227AF7BFF7A1C7971
:10024E0061C003C002C0017B017A0079C490011D18
:10025E00EBF0A3EAF0A3E9F0D001D002D003120E26
:10026E0050900172E0FFEF640460030203E8900116
:10027E0072E4F07E007F0C7DFF7B017A01795012D3
:10028E000D607DFF7F807E3812114A900081E4F070
:10029E00900081E0FFEFC3940C40030203E890004E
:1002AE0081E0FF7E00EF2481FFEE3438FE90008166
:1002BE00E0FD74502DF582E43401F583E0FD12115A
:1002CE004A900081E004F080C70203E890018CE0C0
:1002DE00FFEF30E65490018CE0FFEF54BFFF90012A
:1002EE008CEFF090014FE0FFEF70047F0180027FF2
:1002FE000090014FEFF090014FE0FFEF24FF92923C
:10030E007B017A0179C0121814EF601D7BFF7A1CF5
:10031E00796B9001C0E0FF90011DEFF09001C2E0FB
:10032E00FF90011EEFF0120E50900172E0FFEF648D
:10033E000160030203E8900172E4F07E007F207DED
:10034E00007B017A007982120D60900082743EF07B
:10035E00900083744CF09000847454F07B017A0109
:10036E007950C003C002C0017B017A007985A801D3
:10037E00AC02AD03D001D002D0037E007F0C120878
:10038E003E7B017A007982C003C002C0017B017AF4
:10039E000079C2900192EBF0A3EAF0A3E9F0D0014C
:1003AE00D002D0037D0F12192E7B017A0079C27D07
:1003BE00201227AF7BFF7A1C7961C003C002C001F7
:1003CE007B017A0079C490011DEBF0A3EAF0A3E95A
:1003DE00F0D001D002D003120E503083030201A5DB
:1003EE007B017A0079A27D2012202FEF700302018B
:1003FE00A57B017A0079A2C003C002C0017B017AFD
:10040E000079E2900181EBF0A3EAF0A3E9F0D001CC
:10041E00D002D0037D2012151CEF70030201A57FC0
:10042E000212275E7BFF7A1C797BC003C002C001DB
:10043E009000E2E0FBA3E0FAA3E0F9E92402F9EA76
:10044E003400FA90011DEBF0A3EAF0A3E9F0D0011D
:10045E00D002D003120E509000E2E0FBA3E0FAA30C
:10046E00E0F975820275830012087DFFEF120B8A88
:10047E0004882A063D3E000001A59000E2E0FBA3A1
:10048E00E0FAA3E0F975820375830012087DFFEF91
:10049E00120B8A054A3101A53204AE3F000001A5B8
:1004AE007E007F207D007B017A007982120D6090A4
:1004BE000082742AF09000837431F07B017A017906
:1004CE0042C003C002C0017B017A007984A801AC4E
:1004DE0002AD03D001D002D0037E007F0C12083E85
:1004EE007B017A007982C003C002C0017B017A00D1
:1004FE0079C2900192EBF0A3EAF0A3E9F0D001D01B
:10050E0002D0037D0E12192E7B017A0079C27D2056
:10051E001227AF7BFF7A1C7961C003C002C0017B3A
:10052E00017A0079C490011DEBF0A3EAF0A3E9F083
:10053E00D001D002D003120E500201A59000E2E0CD
:10054E00FBA3E0FAA3E0F9E92404F9EA3400FAC0C7
:10055E0003C002C0017B017A017950A801AC02AD43
:10056E0003D001D002D0037E007F0C12083E7D4ADC
:10057E007F807E3812114A900081E4F0900081E075
:10058E00FFEFC3940C502B900081E0FF7E00EF2410
:10059E0081FFEE3438FE900081E0FD74502DF5821F
:1005AE00E43401F583E0FD12114A900081E004F07D
:1005BE0080CA7E007F207D007B017A007982120D39
:1005CE0060900082742AF09000837432F07B017A7E
:1005DE00007982C003C002C0017B017A0079C2900B
:1005EE000192EBF0A3EAF0A3E9F0D001D002D00320
:1005FE007D0212192E7B017A0079C27D201227AF5F
:10060E007BFF7A1C7961C003C002C0017B017A00B6
:10061E0079C490011DEBF0A3EAF0A3E9F0D001D06C
:10062E0002D003120E500201A50201A50201A590EF
:10063E0000E2E0FBA3E0FAA3E0F975820375830004
:10064E0012087DFFEF120B8A065D4C000001A5908B
:10065E0000E2E0FBA3E0FAA3E0F9758204758300E3
:10066E0012087DFFEF645460030201A59000E7E4D9
:10067E00F07B017A017942C003C002C0019000E212
:10068E00E0FBA3E0FAA3E0F9E92405F9EA3400FA65
:10069E00A801AC02AD03D001D002D0037E007F0CC6
:1006AE00120D3CEF702390014EE0FFEF70047F01BE
:1006BE0080027F0090014EEFF090014EE0FFEF249C
:1006CE00FF92849000E77401F07E007F207D007B16
:1006DE00017A007982120D60900082743EF09000D3
:1006EE0083744CF09000847454F09000E7E0FFEFB8
:1006FE0060047F4E80027F59900085EFF07B017A77
:10070E00007982C003C002C0017B017A0079C290D9
:10071E000192EBF0A3EAF0A3E9F0D001D002D003EE
:10072E007D0412192E7B017A0079C27D201227AF2B
:10073E007BFF7A1C7961C003C002C0017B017A0085
:10074E0079C490011DEBF0A3EAF0A3E9F0D001D03B
:0F075E0002D003120E500201A50201A50201A54F
:01076D002269
:101E7A0002001EE493A3F8E493A34003F68001F260
:101E8A0008DFF48029E493A3F85407240CC8C33369
:101E9A00C4540F4420C8834004F456800146F6DF38
:101EAA00E4800B0102040810204080902882E47E1E
:101EBA00019360BCA3FF543F30E509541FFEE4932D
:101ECA00A360010ECF54C025E060A840B8E493A3F4
:101EDA00FAE493A3F8E493A3C8C582C8CAC583CA1F
:101EEA00F0A3C8C582C8CAC583CADFE9DEE780BED7
:0128BC00001B
:10076E00E709F608DFFA8046E709F208DFFA803E6D
:10077E0088828C83E709F0A3DFFA8032E309F6085A
:10078E00DFFA8078E309F208DFFA807088828C83C2
:10079E00E309F0A3DFFA806489828A83E0A3F60876
:1007AE00DFFA805889828A83E0A3F208DFFA804C50
:1007BE0080D280FA80C680D4806980F28033801027
:1007CE0080A680EA809A80A880DA80E280CA803390
:1007DE0089828A83ECFAE493A3C8C582C8CCC58308
:1007EE00CCF0A3C8C582C8CCC583CCDFE9DEE780D8
:1007FE000D89828A83E493A3F608DFF9ECFAA9F057
:10080E00EDFB2289828A83ECFAE0A3C8C582C8CCAC
:10081E00C583CCF0A3C8C582C8CCC583CCDFEADEC5
:10082E00E880DB89828A83E493A3F208DFF980CC27
:10083E0088F0EF60010E4E60C388F0ED2402B40420
:10084E000050B9F582EB2402B4040050AF232345C7
:06085E0082239007BE7327
:10086400BB010689828A83E0225002E722BBFE0292
:09087400E32289828A83E49322C5
:10087D00BB010CE58229F582E5833AF583E0225030
:10088D0006E92582F8E622BBFE06E92582F8E2227A
:0D089D00E58229F582E5833AF583E4932294
:1008AA00BB010689828A83F0225002F722BBFE012D
:0208BA00F32227
:1008BC00F8BB010DE58229F582E5833AF583E8F072
:1008CC00225006E92582C8F622BBFE05E92582C81E
:0208DC00F22206
:1008DE00EF8DF0A4A8F0CF8CF0A428CE8DF0A42E2E
:0208EE00FE22E8
:1008F000BC000BBE0029EF8DF084FFADF022E4CCEC
:10090000F875F008EF2FFFEE33FEEC33FCEE9DECB4
:10091000984005FCEE9DFE0FD5F0E9E4CEFD22EDFA
:10092000F8F5F0EE8420D21CFEADF075F008EF2F44
:10093000FFED33FD4007985006D5F0F222C398FD35
:050940000FD5F0EA22D2
:10094500C5F0F8A3E028F0C5F0F8E582158270023D
:060955001583E038F022DA
:10095B00A3F8E0C5F025F0F0E5821582700215834F
:06096B00E0C838F0E822AC
:10097100BB0110E58229F582E5833AF583E0F5F0C4
:10098100A3E0225009E92582F886F008E622BBFEA1
:100991000AE92582F8E2F5F008E222E5832AF583E7
:0809A100E993F5F0A3E99322AC
:1009A900F8BB0111E58229F582E5833AF583E8F080
:1009B900E5F0A3F0225009E92582C8F608A6F0223D
:0D09C900BBFE09E92582C8F2E5F008F22224
:1009D60075F008758200EF2FFFEE33FECD33CDCCD8
:1009E60033CCC58233C5829BED9AEC99E58298405B
:1009F6000CF582EE9BFEED9AFDEC99FC0FD5F0D638
:100A0600E4CEFBE4CDFAE4CCF9A88222B800C1B961
:100A16000059BA002DEC8BF084CFCECDFCE5F0CB9F
:100A2600F97818EF2FFFEE33FEED33FDEC33FCEBD8
:100A360033FB10D703994004EB99FB0FD8E5E4F993
:100A4600FA227818EF2FFFEE33FEED33FDEC33FC80
:100A5600C933C910D7059BE99A4007EC9BFCE99A74
:100A6600F90FD8E0E4C9FAE4CCFB2275F010EF2FB9
:100A7600FFEE33FEED33FDCC33CCC833C810D707B9
:100A86009BEC9AE899400AED9BFDEC9AFCE899F8F4
:0E0A96000FD5F0DAE4CDFBE4CCFAE4C8F92287
:100AA400EB9FF5F0EA9E42F0E99D42F0EC6480C8C9
:060AB40064809845F02269
:100ABA00EB9FF5F0EA9E42F0E99D42F0E89C45F092
:010ACA002209
:100ACB00E8600FECC313FCED13FDEE13FEEF13FF09
:030ADB00D8F1222D
:0C0ADE00ECF0A3EDF0A3EEF0A3EFF0228B
:100AEA00A8828583F0D083D082120B01120B0112E7
:100AFA000B01120B01E473E493A3C583C5F0C5830C
:100B0A00C8C582C8F0A3C583C5F0C583C8C582C855
:010B1A0022B8
:100B1B00BB010789828A83020D9E5005E9F8020DFD
:100B2B008CBBFE05E9F8020DC789828A83020DD9B9
:100B3B00BB011A89828A83D0F0D0E0F8D0E0F9D0DB
:100B4B00E0FAD0E0FBE8C0E0C0F0020DBE5016E9C1
:100B5B00F8D083D082D0E0F9D0E0FAD0E0FBC082AD
:100B6B00C083020D95BBFE16E9F8D083D082D0E08E
:0F0B7B00F9D0E0FAD0E0FBC082C083020DD02297
:100B8A00D083D082F8E4937012740193700DA3A3FA
:100B9A0093F8740193F5828883E47374029368600E
:060BAA00EFA3A3A380DF0E
:060BB0008A838982E473D0
:100DE500E508241DF582E43401F583E00508229029
:100DF500011A30070390011DE475F001120DA702D9
:100E050008642000E97F2ED2008018EF540F24904B
:100E1500D43440D4FF30040BEF24BFB41A00500380
:100E25002461FFE50960021509050CE50C70020552
:100E35000B30070E90011AE475F001120DA7EF02B1
:100E450008AA0229827403D2078003E4C207F508C1
:100E550090011A120DBEE4F509F50BF50CE50960D4
:100E6500077F20120E2880F5750AFFC201C200C255
:100E750002C203C205C206C208120DF4FF700D308E
:100E850007057F00120E39AF0CAE0B22B4255FC2E9
:100E9500D5C204120DF4FF24D0B40A00501A75F01F
:100EA5000A780930D50508B6FF0106C6A426F6203E
:100EB500D5047002D20380D924CFB41A00EF5004B0
:100EC500C2E5D20402103AD20180C6D20080C0D257
:100ED5000280BCD2D580BAD20580B47F20120E28FC
:100EE5002002077401B5090040F1120DE5FF120E4D
:100EF50028020E62D208D2068095120DE5FB120D6E
:100F0500E5FA120DE5F94A4B7006790B7A117BFF6C
:100F150020022EE509602A7E008E82758300120864
:100F25007D60060EEE650A70F0C2D5EBC0E0EAC042
:100F3500E0E9C0E0EE121081D0E0F9D0E0FAD0E0AF
:100F4500FB120864FF60AAEBC0E0EAC0E0E9C0E07C
:100F5500120E28D0E02401F9D0E03400FAD0E0FBED
:100F6500E50A0460DCD50AD980877BFF7A10797D94
:100F7500D202809C791080027908C206C2088008D6
:100F8500D2D5790A8004790AC2D5E50A047002F53A
:100F95000AE4FAFDFEFF120DE5FC7B0820011312A1
:100FA5000DE5FD7B1030000A120DE5FE120DE5FF83
:100FB5007B20EC3382D592D55013C3E43000069FD5
:100FC500FFE49EFEE42001039DFDE49CFCE4CBF8D8
:100FD500C201EC700CCFCECDCCE824F8F870F380CC
:100FE50017C3EF33FFEE33FEED33FDEC33FCEB338C
:100FF500FB994002FB0FD8E9EB300105F8D0E0C4BE
:1010050048B201C0E00AEC4D4E4F78207B0070C21B
:10101500EAB50A0040BCC0E0121083D0F0D0E02051
:101025000104C4C0E0C4B201C0F0120E11D0F0D565
:10103500F0EB020E62120B8A0EFF530F79580ED099
:101045004C0ECC420F7D4F0F85440F85490EE5436D
:081055000F8B550F6F460F6F62
:10105D00450F6F47112B500ED42D0ED82E0EFB2B96
:10106D000EDC230EF92011142A0E944800000EF305
:10107D003F3F3F00790AA2D5200314300509B9106E
:10108D00020404B9080104A2D5200602500104206F
:10109D0002689202B509005034C0E07F2030031978
:1010AD007F30A20272067205500F1210DAC202C210
:1010BD0006C205C2087F30800F300503E9C0E0127B
:1010CD000E28300503D0E0F9D0E0B509CC30051776
:1010DD007F30B9100C120E287F583004077F7880AE
:1010ED0003B90803120E283002057F2D020E287F4A
:1010FD00202008F87F2B2006F322920280CF286E45
:10110D00756C6C2900D201120DE53001F8C2017821
:10111D000930D50108F6020E942D50434958120D91
:10112D00E52403B405004001E490112693120E1935
:0D113D00743A120E19D203750904020F79DD
:100BB600E3F5F009E208B5F06BDFF58067E3F5F0E1
:100BC60009E608B5F05EDFF5805A87F009E608B554
:100BD600F052DFF6804E87F009E208B5F046DFF600
:100BE600804288828C8387F009E0A3B5F036DFF671
:100BF600803288828C8387F009E493A3B5F025DFE1
:100C0600F5802188828C83E3F5F009E0A3B5F01422
:100C1600DFF5801088828C83E3F5F009E493A3B5B1
:100C2600F002DFF4020CE5808780E9809080D480B2
:100C36003E8015806E807E809D80B7808D80A380EB
:100C4600518074803C020CF189828A83ECFAE49329
:100C5600F5F0A3C8C582C8CCC583CCE493A3C8C5A8
:100C660082C8CCC583CCB5F076DFE3DEE18070893F
:100C7600828A83E493F5F0A3E208B5F062DFF4809C
:100C86005E89828A83E0F5F0A3E608B5F051DFF5C8
:100C9600804D89828A83E0F5F0A3E208B5F040DF53
:100CA600F5803C89828A83E493F5F0A3E608B5F0E3
:100CB6002EDFF4802A8002805789828A83ECFAE448
:100CC60093F5F0A3C8C582C8CCC583CCE0A3C8C53C
:100CD60082C8CCC583CCB5F006DFE4DEE280007FB7
:100CE600FFB5F0020F2240027F012289828A83EC3F
:100CF600FAE0F5F0A3C8C582C8CCC583CCE0A3C88A
:100D0600C582C8CCC583CCB5F0D5DFE5DEE380CFA0
:100D160089828A83ECFAE0F5F0A3C8C582C8CCC5FF
:100D260083CCE493A3C8C582C8CCC583CCB5F0AF49
:100D3600DFE4DEE280A988F0EF60010E4E60ABEDE5
:100D46002402B404005098F582EB2402B404005047
:0A0D56008E2323458223900C2D7399
:100D6000EF4E6012EF60010EEDBB010B89828A83AA
:100D7000F0A3DFFCDEFA2289F05007F709DFFCA9B7
:0C0D8000F022BBFEFCF309DFFCA9F0220E
:090D8C00E6FB08E6FA08E6F9228C
:090D9500EBF608EAF608E9F62283
:090D9E00E0FBA3E0FAA3E0F92256
:100DA700F8E0FBA3A3E0F925F0F0E58215827002D5
:070DB7001583E0FA38F02279
:090DBE00EBF0A3EAF0A3E9F02236
:090DC700E2FB08E2FA08E2F9225D
:090DD000EBF208EAF208E9F22254
:0C0DD900E493FB740193FA740293F92276
:10298200EFB40A07740D12298D740A309811A899B0
:10299200B8130CC2983098FDA899C298B811F630B5
:0729A20099FDC299F599228D
:00000001FF
